:1000000019C018951895189518951895189518955C
:1000100018951895189518951895DDC01895189588
:100020001895189518951895189518951895189568
:10003000189518958FEF8DBFC0EEE8ED4E2E82E03B
:100040008EBFD2E0F2E05F2EEEEFF1E0A0E0B1E093
:10005000A89584B7082E877F84BF88E1992780936D
:1000600060009093600088278D933197E9F783E3D0
:100070008093C40080E08093C50088E18093C10034
:100080006624209A219A229A289829982A9887E803
:1000900080937A0080EC80937C00279A2F9A269890
:1000A000259A2D987CD080E08093800084E0809316
:1000B0008100789480916F00816080936F0084E06C
:1000C000809381002D9AE1E0F0E006D170917A00F2
:1000D000706870937A0000917C00007F006000934C
:1000E0007C0018D1A0E0B1E08D939C93A0ECB2E02D
:1000F000E0E0F1E054D1D8D0E5D02D98A0E0B1E017
:100100000D911C91083552E0150714F009F001C05B
:1001100005C082E0E4ECF9E0A5E221D1A0E0B1E085
:100120000D911C91083552E0150781E014F009F09B
:1001300080E08F93A0E0B1E00D911C91063252E077
:10014000150780E014F009F081E09F91892388234E
:1001500009F405C081E0E4ECF9E0A5E200D1A0E0FB
:10016000B1E00D911C91063252E0150714F009F030
:1001700005C080E0E4ECF9E0A5E2F1D0A0E0B1E058
:100180000D911C910C3152E015070CF401C001C017
:1001900059C081E083BF889595CFF894FFCFE0E404
:1001A000F4E08AD08FD0E4E5F4E086D08BD08AD01A
:1001B000289A82E390E09FD0299A82E390E09BD036
:1001C00028982A9A82E390E096D0299882E390E0DA
:1001D00092D02A9808950F921F922F923F924F9299
:1001E0005F927F92AF92BF920F931F932F933F9393
:1001F0004F935F936F937F938F939F93AF93BF932F
:10020000CF93DF93EF93FF938FB78F938F918FBF30
:10021000FF91EF91DF91CF91BF91AF919F918F911E
:100220007F916F915F914F913F912F911F910F910E
:10023000BF90AF907F905F904F903F902F901F9016
:100240000F9018952F98E1E0F0E046D0A2E0B1E0E1
:1002500024D00027A3E2B0E08C9186FB0EF401E0ED
:1002600040E0041709F008C02F9A80E090E0A2E077
:10027000B1E08D939C9326CFA2E0B1E00D911C914B
:10028000003A5CE8150709F0DDCF2F9A80E090E096
:10029000A2E0B1E08D939C9315CFED91FC91EF5FBF
:1002A000FF4FFC93EE930895A0ECB2E08D9188236C
:1002B00011F00BD0FBCF089544D0802D11F005D064
:1002C000FBCF08958DE001D08AE00090C00005FECC
:1002D000FCCF8093C600089588EE93E00CD0319750
:1002E000D9F708953197F1F70895689462F8089561
:1002F000E89462F80895EF93FF93EE27E82BE92B3B
:1003000031F0EAEFF0E03197F1F70197D1F7FF9183
:10031000EF91089570917A00706470937A00009064
:100320007A0006FCFCCF70917A00706470937A00BA
:1003300000907A0006FCFCCF8091780090917900C3
:100340000895C89531960020089591E0882321F002
:100350008894991F8A95E9F7892F90950895BB276E
:10036000F4DF9C9198279C933197F1F798279C9301
:100370000895000F111F221F331F08950095109537
:10038000209530950F5F1F4F2F4F3F4F08950191DC
:1003900010810EC001911191219130810BC001910A
:1003A000108117FF05C03FEF2FEF04C00081112718
:1003B0002227332737FF03C0E1DF8DE28D93CF93F0
:1003C000DF93CF92DF92EF92AA24BB24CC24DD24CA
:1003D000EE2440E2CAE0DD2755E093E38881890FEF
:1003E00087FD9F7083FD907F891B89935A95A9F79C
:1003F000C0DFAA1CBB1CCC1CDD1CEE1C4A9551F7AF
:10040000E894EFE0FF2782910ED0EB30E0F71EF08A
:1004100068948A2D0CD088278D93EF90DF90CF9031
:10042000DF91CF910895982F829501D0892F8F70F9
:10043000805D26F0803309F4089568948D930895C3
:100440007C43686172676520436F6E74726F6C6C79
:1004500065727C007C41565270726F6A6563742EBF
:080460007275202020207C00B1
:00000001FF
